:020000040800F2
:1000000000000520C1100008BD0F0008C50F000842
:10001000CD0F0008D50F0008DD0F0008000000001C
:10002000000000000000000000000000E50F0008D4
:10003000F30F000800000000011000080F10000876
:100040001111000811110008111100081111000808
:1000500011110008111100081111000811110008F8
:1000600011110008111100081111000811110008E8
:1000700011110008111100081111000811110008D8
:1000800011110008111100081111000811110008C8
:1000900011110008111100081111000811110008B8
:1000A00011110008111100081111000811110008A8
:1000B0001111000811110008111100081111000898
:1000C0001111000811110008111100081111000888
:1000D0001111000811110008111100081111000878
:1000E0001111000811110008111100081111000868
:1000F0001111000811110008111100081111000858
:100100001111000811110008111100081111000847
:100110001D1000081111000811110008111100082C
:100120001111000811110008111100081111000827
:100130001111000811110008111100081111000817
:100140001111000811110008111100081111000807
:1001500011110008111100081111000811110008F7
:1001600011110008111100081111000811110008E7
:100170001111000811110008000000001111000801
:1001800011110008111100081111000811110008C7
:1001900011110008111100080000000011110008E1
:1001A00011110008111100080000000000000000FB
:1001B00011110008000000000000000011110008EB
:1001C0001111000811110008111100081111000887
:0801D0001111000811110008D3
:1001E00010B5054C237833B9044B13B10448AFF371
:1001F00000800123237010BD7C000020000000005F
:100200003045000808B5034B1BB103490348AFF361
:10021000008008BD0000000080000020304500087C
:10022000034613F8012B002AFBD1181A0138704736
:1002300001F0FF01102A2BDB10F0070F08D010F897
:10024000013B013A8B422DD010F0070F42B3F6D19B
:10025000F0B441EA012141EA014122F007047FF0B4
:1002600000070023F0E80256083C85EA010586EA0B
:10027000010685FA47F5A3FA87F586FA47F6A5FA47
:1002800087F68EB9EED1F0BC01F0FF0102F0070253
:1002900032B110F8013B013A83EA010313B1F8D1FE
:1002A0000020704701387047002D06BF35460338DF
:1002B000073815F0010F07D1013015F4807F02BF18
:1002C000013015F4C03F0130F0BC0138704700BF69
:1002D00053B94AB9002908BF00281CBF4FF0FF31AD
:1002E0004FF0FF3000F06AB9ADF1080C6DE904CEB3
:1002F00000F006F8DDF804E0DDE9022304B0704701
:100300002DE9F047089D0C46002B4ED194468C45B4
:100310008646B2FA82F262D94AB1C2F12003914014
:1003200020FA03F30CFA02FC194300FA02FE4FEA2A
:100330001C471FFA8CF6B1FBF7F44FEA1E4307FB8C
:10034000141143EA014304FB06F199420AD91CEB5C
:10035000030304F1FF3080F01281994240F20F81D3
:10036000023C6344591A1FFA8EF3B1FBF7F007FB06
:10037000101143EA014300FB06F69E420AD91CEB2A
:10038000030300F1FF3180F0FC809E4240F2F980CF
:10039000634402389B1B40EA044000211DB1D34056
:1003A0000022C5E90032BDE8F0878B4205D90DB1C6
:1003B000C5E9000100210846F5E7B3FA83F10029F9
:1003C00046D1A34202D39042C0F0F080861A64EB7B
:1003D00003030120002DE6D0C5E90063E3E7002A0E
:1003E00040F09080A1EB0C044FEA1C481FFA8CF7F8
:1003F0000121B4FBF8F64FEA1E4308FB164443EA1A
:10040000044307FB06F0984208D91CEB030306F1EE
:10041000FF3402D2984200F2CD8026461C1A1FFA01
:100420008EF3B4FBF8F008FB104443EA044300FBEE
:1004300007F79F4208D91CEB030300F1FF3402D2F7
:100440009F4200F2B0802046DB1B40EA0640A5E751
:10045000C1F120068B4022FA06F71F4320FA06FC62
:1004600004FA01F343EA0C03F44000FA01F8380CF3
:100470004FEA1349B4FBF0FE1FFA87FC00FB1E4451
:1004800049EA04440EFB0CF9A14502FA01F20AD92B
:100490003C190EF1FF3A80F08480A14540F2818042
:1004A000AEF1020E3C44A4EB09041FFA83F9B4FB3D
:1004B000F0F300FB134449EA044403FB0CFCA4459D
:1004C00007D93C1903F1FF3067D2A44565D9023B37
:1004D0003C4443EA0E40A0FB0293A4EB0C049C4274
:1004E000CE469C4651D34ED055B1B8EB0E0364EBCB
:1004F0000C0404FA06F6CB401E43CC40C5E9006468
:10050000002150E7C2F1200320FA03F10CFA02FCAB
:1005100024FA03F394400C434FEA1C4800FA02FE0D
:100520001FFA8CF7B3FBF8F008FB1031230C43EAF9
:10053000014300FB07F1994208D91CEB030300F1CA
:10054000FF362CD299422AD9023863445B1AA4B2EE
:10055000B3FBF8F108FB113344EA034401FB07F352
:10056000A34208D91CEB040401F1FF3613D2A342C5
:1005700011D902396444E41A41EA004139E70446DA
:10058000F0E6084606E7C845AED2B9EB020E63EBCB
:10059000070C0138A8E73146EDE7034699E73046F6
:1005A000D4E7D6467FE7634402384DE70646234644
:1005B00008460FE7023E634430E700BF704700BFC4
:1005C00080B485B000AFF860B9601346FB80FB686B
:1005D00000221A80FB6800225A80FB6800229A8061
:1005E000FB68BA689A60FB68FA88DA80FB680022C8
:1005F0001A7300BF1437BD465DF8047B704780B5A1
:1006000086B000AFF860B9601346FB80F86800F070
:10061000E6F803467B82FB885A1CB7F912309A42EF
:1006200042DAFB685B881A46FB8813440133FA6898
:10063000D288934207DBFB685B881A46FB68DB883D
:10064000023B9A4230DBFB881946F86800F00EF94D
:10065000FB689B68FA6852881344FA88B9681846A0
:1006600000F0E8F8FB685A88FB8813449AB2FB68EC
:100670005A80FB685A88FB68DB889A4202D1FB6883
:1006800000225A80FB689B8801339AB2FB689A80EB
:10069000FB685A88FB681B889A4202D1FB680122DA
:1006A0001A7300237B6150E0FB88DA1CB7F9123023
:1006B0009A4247DAFB68DA88FB685B88D31A9BB2F8
:1006C000023B3B823B8A1946F86800F0CFF8FB6892
:1006D0009B68FA68528813443A8AB968184600F051
:1006E000A9F8FB6800225A80FA883B8AD31AFB805B
:1006F000FB881946F86800F0B9F8FB689B68FA684F
:10070000528898183B8ABA681344FA88194600F050
:1007100091F8FB685A88FB8813449AB2FB685A80A8
:10072000FB689B8802339AB2FB689A80FB685A8800
:10073000FB681B889A4202D1FB6801221A730023CE
:100740007B6102E04FF0FF337B617B69184618370D
:10075000BD4680BD80B487B000AFF860B9607A60F4
:10076000FB689B88002B03D14FF0FF337B612FE0A8
:10077000FB681B887B82FB689A687B8A591C79829C
:1007800013441B781B023B82FB68DB887A8A9A42FF
:1007900001D100237B82FB689A687B8A591C79828D
:1007A00013441B781A463B8A13433B82FB68DB8861
:1007B0007A8A9A4201D100237B82FB689A687B8AFD
:1007C0001A44BB681A607B683A8A1A8000237B61EE
:1007D0007B6918461C37BD465DF8047B704780B4C2
:1007E00085B000AF78607B685A887B681B889A4226
:1007F0000BD37B68DA887B6819887B685B88CB1AA7
:100800009BB213449BB2FB8106E07B681A887B682D
:100810005B88D31A9BB2FB817B681B7B012B01D1C8
:100820000023FB81B7F90E3018461437BD465DF83A
:10083000047B704780B485B000AFF860B9601346A0
:10084000FB8007E0BA68531CBB60FB68591CF96069
:1008500012781A70FB885A1EFA80002BF2D100BF62
:1008600000BF1437BD465DF8047B704790B482B07A
:1008700000AF78600B467B807B881B0A98B27B6850
:100880009A687B685B88591C8CB279684C801344E9
:10089000C2B21A707B685A887B68DB889A4202D1A0
:1008A0007B6800225A807B689A687B685B88591C49
:1008B00088B27968488013447A88D2B21A707B680B
:1008C0005A887B68DB889A4202D17B6800225A8072
:1008D00000BF0837BD4690BC7047000080B582B0AD
:1008E00000AF0023FB714FF4006204490448FFF796
:1008F00067FEFB7918460837BD4680BDA80000207A
:100900009800002080B582B000AF0346FB71FB79F0
:10091000012B03D1094B01221A700BE0074B002277
:100920001A70074B01221A704FF4006205490648FD
:10093000FFF746FE00BF0837BD4680BDA80C00206B
:1009400000000020A80000209800002080B483B0A0
:1009500000AF0346FB71FB79FF2B02D0044AFB7901
:10096000137000BF0C37BD465DF8047B704700BFB5
:100970001C0000200EB480B585B000AF0346FB71AB
:100980001F4B1B78FA799A4233D31E4B1B78012BED
:100990002FD10023FB60FB791B4A52F823301B4AFE
:1009A0004FF480611A4803F0D5F8F86007F120038E
:1009B000BB60FB68164A9818FB68C3F58061BB688A
:1009C000FA6903F027F9F8601148FFF729FC03469C
:1009D0001A460F4B13440F4A1188927819809A7067
:1009E0000B48FFF71DFC03469BB21946084800F070
:1009F00013F800BF1437BD46BDE8804003B0704710
:100A00001C000020A80C00200400002078450008ED
:100A1000A80800208045000880B586B000AF786047
:100A20000B467B807B881A4679681048FFF7E7FD04
:100A300078617B69002B15D10D4B1B78DBB2012B44
:100A400010D10B4B00221A7007F10E0207F11003B0
:100A500019460648FFF77EFE3B69FA8919460548A4
:100A600002F064F900BF1837BD4680BD9800002031
:100A700000000020000D002080B500AF00F04AFB10
:100A800000F03AF800F00CF900F0A0F800F0DEF801
:100A9000FFF724FF0346002B01D000BFFDE7012034
:100AA000FFF730FF104B1B781846FFF74FFF0F4939
:100AB0000120FFF75FFF00F099F90221042000F008
:100AC000A1F9BF21062000F09DF94FF4806108488C
:100AD00000F0EEFE03461A46064B1A70642000F042
:100AE0008BFB00BFF1E700BF1D000020844500081C
:100AF00000000240480D002080B594B000AF07F11F
:100B00001C0334220021184603F092F807F1080371
:100B100000221A605A609A60DA601A6100237B60D2
:100B2000284B1B6C274A43F080531364254B1B6CE6
:100B300003F080537B607B6800233B60224B1B6883
:100B4000214A43F4404313601F4B1B6803F44043A6
:100B50003B603B680223FB610123BB621023FB6205
:100B600002237B630023BB630823FB6364233B6492
:100B700002237B640223BB640223FB6407F11C0392
:100B8000184601F0FFFD0346002B01D000F028F9C4
:100B90000F23BB600223FB6000233B614FF48053B3
:100BA0007B610023BB6107F108030321184601F0B4
:100BB000C9FB0346002B01D000F012F900BF5037EB
:100BC000BD4680BD003802400070004080B500AFD7
:100BD0001B4B1C4A1A601A4B1B4A5A60184B0022C6
:100BE0009A60174B0022DA60154B4FF480421A616D
:100BF000134B00225A61124B00229A61104B0022C3
:100C0000DA610F4B00221A620D4800F083FE0346A2
:100C1000002B01D000F0E4F80021094801F017FB97
:100C20000346002B01D000F0DBF80021044801F05E
:100C30004AFB0346002B01D000F0D2F800BF80BD74
:100C4000AC0C002000580040A086010080B500AF29
:100C5000114B124A1A60104B4FF4E1325A600E4B9E
:100C600000229A600C4B0022DA600B4B00221A61C2
:100C7000094B0C225A61084B00229A61064B002254
:100C8000DA61054802F002F80346002B01D000F0BB
:100C9000A7F800BF80BD00BF000D0020004C004041
:100CA00080B58AB000AF07F1140300221A605A60C1
:100CB0009A60DA601A6100233B61454B1B6B444A22
:100CC00043F001031363424B1B6B03F001033B61D1
:100CD0003B690023FB603E4B1B6B3D4A43F008031E
:100CE00013633B4B1B6B03F00803FB60FB680023A3
:100CF000BB60374B1B6B364A43F020031363344B06
:100D00001B6B03F02003BB60BB6800237B60304B90
:100D10001B6B2F4A43F0040313632D4B1B6B03F033
:100D200004037B607B6800233B60294B1B6B284AD4
:100D300043F002031363264B1B6B03F002033B607B
:100D40003B6800224FF40041224800F0C9FD002218
:100D50004FF48061204800F0C3FD4FF400437B61F5
:100D60000123BB610023FB6100233B6207F11403F5
:100D70001946184800F008FC4FF480637B6100239B
:100D8000BB610023FB6107F114031946114800F011
:100D9000FBFB4FF480637B610123BB610023FB619C
:100DA00000233B6207F1140319460B4800F0ECFBEB
:100DB00001237B610023BB610023FB6107F1140366
:100DC0001946064800F0E0FB00BF2837BD4680BD4D
:100DD00000380240000002400014024000080240B7
:100DE00080B400AF72B600BF00BFFDE780B500AFB2
:100DF0000721002000F006F8012000F0FDF900BFF7
:100E000080BD000080B586B002AF03460A46FB7184
:100E10001346BB71FB793B73BB797B7307F10C0203
:100E20004FF0FF33009302236421034800F0B6FE25
:100E300000BF1037BD4680BDAC0C002080B483B02D
:100E400000AF00237B60104B5B6C0F4A43F4804380
:100E500053640D4B5B6C03F480437B607B68002321
:100E60003B60094B1B6C084A43F080531364064BEC
:100E70001B6C03F080533B603B6800BF0C37BD46E2
:100E80005DF8047B704700BF0038024080B58AB02F
:100E900000AF786007F1140300221A605A609A606C
:100EA000DA601A617B681B68194A93422CD10023CF
:100EB0003B61184B1B6B174A43F002031363154B3E
:100EC0001B6B03F002033B613B694FF440637B61A2
:100ED0001223BB610023FB6103233B6204237B627B
:100EE00007F1140319460C4800F04EFB0023FB6089
:100EF000084B1B6C074A43F480031364054B1B6CBF
:100F000003F48003FB60FB6800BF2837BD4680BD4B
:100F100000580040003802400004024080B58AB00A
:100F200000AF786007F1140300221A605A609A60DB
:100F3000DA601A617B681B681D4A934233D1002333
:100F40003B611C4B1B6C1B4A43F400231364194B7D
:100F50001B6C03F400233B613B690023FB60154BD2
:100F60001B6B144A43F008031363124B1B6B03F013
:100F70000803FB60FB6803237B610223BB61002342
:100F8000FB6103233B620B237B6207F114031946C9
:100F9000094800F0F9FA00220421342000F02BFA6D
:100FA000342000F044FA00BF2837BD4680BD00BFA2
:100FB000004C004000380240000C024080B400AFFA
:100FC00000BFFDE780B400AF00BFFDE780B400AF15
:100FD00000BFFDE780B400AF00BFFDE780B400AF05
:100FE00000BFFDE780B400AF00BFBD465DF8047BE5
:100FF000704780B400AF00BFBD465DF8047B70470A
:1010000080B400AF00BFBD465DF8047B704780B57B
:1010100000AF00F0D1F800BF80BD000080B500AF88
:10102000024801F0B9FE00BF80BD00BF000D0020E6
:1010300080B586B000AF7860144A154BD31A7B6137
:101040007B693B61134B1B68002B02D1114B124A89
:101050001A60104B1A687B6813443A699A4207D2A7
:1010600002F0EEFD03460C221A604FF0FF3309E058
:10107000084B1B68FB60074B1A687B681344054AE2
:101080001360FB6818461837BD4680BD0000052078
:10109000000400004C0D0020A00E002080B400AF22
:1010A000064BD3F88830054A43F47003C2F8883001
:1010B00000BFBD465DF8047B704700BF00ED00E057
:1010C000DFF834D0FFF7EAFF0C480D490D4A002342
:1010D00002E0D458C4500433C4188C42F9D30A4AED
:1010E0000A4C002301E013600432A242FBD302F059
:1010F000ADFDFFF7C1FC7047000005200000002097
:101100007C000020FC4500087C0000209C0E002094
:10111000FEE7000080B500AF0E4B1B680D4A43F49C
:10112000007313600B4B1B680A4A43F4806313601F
:10113000084B1B68074A43F480731360032000F0D8
:101140004FF90F2000F008F8FFF778FE002318464B
:1011500080BD00BF003C024080B582B000AF786027
:10116000124B1A68124B1B7819464FF47A73B3FB73
:10117000F1F3B2FBF3F3184600F067F90346002BD6
:1011800001D001230EE07B680F2B0AD8002279687A
:101190004FF0FF3000F02FF9064A7B681360002300
:1011A00000E0012318460837BD4680BD200000201E
:1011B000280000202400002080B400AF064B1B78DC
:1011C0001A46064B1B681344044A136000BFBD4611
:1011D0005DF8047B704700BF28000020500D002000
:1011E00080B400AF034B1B681846BD465DF8047B16
:1011F000704700BF500D002080B584B000AF78600C
:10120000FFF7EEFFB8607B68FB60FB68B3F1FF3F60
:1012100005D00A4B1B781A46FB681344FB6000BFDD
:10122000FFF7DEFF0246BB68D31AFA689A42F7D886
:1012300000BF00BF1037BD4680BD00BF28000020A2
:1012400080B485B000AF78607B6803F00703FB6073
:101250000C4BDB68BB60BA684FF6FF031340BB6002
:10126000FB681A02BB68134343F0BF6343F40033C7
:10127000BB60044ABB68D36000BF1437BD465DF84D
:10128000047B704700ED00E080B400AF044BDB68E6
:101290001B0A03F007031846BD465DF8047B704740
:1012A00000ED00E080B483B000AF0346FB7197F916
:1012B0000730002B0BDBFB7903F01F02074997F97E
:1012C00007305B09012000FA02F241F8232000BF39
:1012D0000C37BD465DF8047B704700BF00E100E0BD
:1012E00080B483B000AF03463960FB7197F90730D3
:1012F000002B0ADB3B68DAB20C4997F90730120180
:10130000D2B20B4483F800230AE03B68DAB2084902
:10131000FB7903F00F03043B1201D2B20B441A769F
:1013200000BF0C37BD465DF8047B704700E100E06C
:1013300000ED00E080B489B000AFF860B9607A6079
:10134000FB6803F00703FB61FB69C3F10703042B90
:1013500028BF0423BB61FB690433062B02D9FB6958
:10136000033B00E000237B614FF0FF32BB6902FAD0
:1013700003F3DA43BB681A407B699A404FF0FF31B0
:101380007B6901FA03F3D9437B680B40134318468A
:101390002437BD465DF8047B7047000080B582B0FD
:1013A00000AF78607B68013BB3F1807F01D30123FC
:1013B0000FE00A4A7B68013B53600F214FF0FF307A
:1013C000FFF78EFF054B00229A60044B07221A603C
:1013D000002318460837BD4680BD00BF10E000E07E
:1013E00080B582B000AF78607868FFF729FF00BF52
:1013F0000837BD4680BD80B586B000AF0346B960F2
:101400007A60FB7300237B61FFF73EFF78617A68A7
:10141000B9687869FFF78EFF024697F90F301146D9
:101420001846FFF75DFF00BF1837BD4680BD80B589
:1014300082B000AF0346FB7197F907301846FFF7FB
:1014400031FF00BF0837BD4680BD80B582B000AF18
:1014500078607868FFF7A2FF034618460837BD4654
:1014600080BD80B584B000AF78607B689B6DFB6009
:10147000FFF7B6FEB8607B6893F83530DBB2022B1D
:1014800008D07B6880225A657B68002283F834206C
:10149000012352E07B681B681A687B681B6822F096
:1014A00016021A607B681B685A697B681B6822F009
:1014B00080025A617B681B6C002B03D17B689B6C9C
:1014C000002B07D07B681B681A687B681B6822F0BA
:1014D00008021A607B681B681A687B681B6822F028
:1014E00001021A6013E0FFF77BFE0246BB68D31AC5
:1014F000052B0CD97B6820225A657B68032283F870
:1015000035207B68002283F83420032315E07B68B4
:101510001B681B6803F00103002BE4D17B68DB6DC3
:101520003F229A40FB689A607B68012283F835204D
:101530007B68002283F83420002318461037BD460C
:1015400080BD80B483B000AF78607B6893F835309D
:10155000DBB2022B04D07B6880225A6501230CE0A9
:101560007B68052283F835207B681B681A687B68D6
:101570001B6822F001021A60002318460C37BD4692
:101580005DF8047B7047000080B489B000AF7860DC
:10159000396000237B6100233B610023BB61002392
:1015A000FB6165E10122FB6902FA03F37B613B68A1
:1015B0001B687A6913403B613A697B699A4240F043
:1015C00054813B685B6803F00303012B05D03B6843
:1015D0005B6803F00303022B30D17B689B68BB611F
:1015E000FB695B00032202FA03F3DB43BA69134091
:1015F000BB613B68DA68FB695B0002FA03F3BA6916
:101600001343BB617B68BA699A607B685B68BB61A6
:101610000122FB6902FA03F3DB43BA691340BB61A1
:101620003B685B681B0903F00102FB6902FA03F3E4
:10163000BA691343BB617B68BA695A603B685B68EF
:1016400003F00303032B17D07B68DB68BB61FB69E6
:101650005B00032202FA03F3DB43BA691340BB6168
:101660003B689A68FB695B0002FA03F3BA691343AB
:10167000BB617B68BA69DA603B685B6803F00303AF
:10168000022B23D1FB69DA087B68083253F8223039
:10169000BB61FB6903F007039B000F2202FA03F30F
:1016A000DB43BA691340BB613B681A69FB6903F00D
:1016B00007039B0002FA03F3BA691343BB61FB699A
:1016C000DA087B680832B96943F822107B681B6826
:1016D000BB61FB695B00032202FA03F3DB43BA69D7
:1016E0001340BB613B685B6803F00302FB695B006E
:1016F00002FA03F3BA691343BB617B68BA691A60E3
:101700003B685B6803F44033002B00F0AE8000239D
:10171000FB605D4B5B6C5C4A43F4804353645A4B03
:101720005B6C03F48043FB60FB68584AFB699B08D1
:10173000023352F82330BB61FB6903F003039B00C3
:101740000F2202FA03F3DB43BA691340BB617B68E3
:101750004F4A934225D07B684E4A93421FD07B6804
:101760004D4A934219D07B684C4A934213D07B6810
:101770004B4A93420DD07B684A4A934207D07B681C
:10178000494A934201D106230CE007230AE00523CE
:1017900008E0042306E0032304E0022302E001231F
:1017A00000E00023FA6902F0030292009340BA6954
:1017B0001343BB613549FB699B080233BA6941F8A1
:1017C00023203A4B9B68BB613B69DB43BA691340FA
:1017D000BB613B685B6803F48013002B03D0BA69DC
:1017E0003B691343BB61314ABB6993602F4BDB6894
:1017F000BB613B69DB43BA691340BB613B685B6813
:1018000003F40013002B03D0BA693B691343BB6197
:10181000264ABB69D360254B5B68BB613B69DB43F0
:10182000BA691340BB613B685B6803F40033002B6B
:1018300003D0BA693B691343BB611C4ABB6953605F
:101840001A4B1B68BB613B69DB43BA691340BB6140
:101850003B685B6803F48033002B03D0BA693B69B3
:101860001343BB61114ABB691360FB690133FB6120
:10187000FB690F2B7FF696AE00BF00BF2437BD4635
:101880005DF8047B704700BF00380240003801401B
:10189000000002400004024000080240000C024028
:1018A000001002400014024000180240003C0140B9
:1018B00080B485B000AF78600B467B807B681A6986
:1018C0007B881340002B02D00123FB7301E000232F
:1018D000FB73FB7B18461437BD465DF8047B7047ED
:1018E00080B483B000AF78600B467B8013467B707A
:1018F0007B78002B03D07A887B689A6103E07B8831
:101900001A047B689A6100BF0C37BD465DF8047B02
:101910007047000080B584B000AF78607B68002B12
:1019200001D101232BE17B6893F83D30DBB2002B22
:1019300006D17B68002283F83C207868FFF7A6FA7E
:101940007B68242283F83D207B681B681A687B68CB
:101950001B6822F001021A607B681B681A687B68AA
:101960001B6842F400421A607B681B681A687B6837
:101970001B6822F400421A6000F0DCFEF8607B680D
:101980005B68814A934207D8FB68804A934294BFC0
:1019900001230023DBB206E0FB687D4A934294BF3B
:1019A00001230023DBB2002B01D00123E7E0FB6819
:1019B000784AA2FB03239B0CBB607B681B685B68B7
:1019C00023F03F017B681B68BA680A435A607B6852
:1019D0001B681B6A23F03F017B685B686A4A93427D
:1019E00002D8BB68013309E0BB684FF4967202FB72
:1019F00003F3694AA2FB03239B0901337A68126847
:101A00000B4313627B681B68DB6923F44F4222F0AF
:101A1000FF027B685B685C498B4219D8FB68591EE2
:101A20007B685B685B00B1FBF3F3591C40F6FC7309
:101A30000B40002B0AD0FB68591E7B685B685B007B
:101A4000B1FBF3F30133C3F30B0351E004234FE085
:101A50007B689B68002B11D1FB68581E7B68596816
:101A60000B465B000B44B0FBF3F30133C3F30B03F2
:101A7000002B0CBF01230023DBB212E0FB68581ED1
:101A80007B6859680B469B000B4499000B44B0FBE4
:101A9000F3F30133C3F30B03002B0CBF012300232B
:101AA000DBB2002B01D0012322E07B689B68002B76
:101AB0000ED1FB68581E7B6859680B465B000B44CF
:101AC000B0FBF3F30133C3F30B0343F400430FE024
:101AD000FB68581E7B6859680B469B000B449900B5
:101AE0000B44B0FBF3F30133C3F30B0343F4404364
:101AF000796809681343CB617B681B681B6823F016
:101B0000C0017B68DA697B681B6A1A437B681B68C3
:101B10000A431A607B681B689B6823F4034323F025
:101B2000FF037A6811697A68D26811437A6812688B
:101B30000B4393607B681B68DB6823F0FF017B68C5
:101B40005A697B689B691A437B681B680A43DA60A1
:101B50007B681B681A687B681B6842F001021A6088
:101B60007B6800221A647B68202283F83D207B6812
:101B700000221A637B68002283F83E200023184667
:101B80001037BD4680BD00BFA08601007F841E00C7
:101B9000FF083D0083DE1B43D34D621080B588B043
:101BA00002AFF8607A601A460B467B8113463B8190
:101BB000FFF716FB7861FB6893F83D30DBB2202B12
:101BC00040F0E0807B690093192301227049F86896
:101BD00000F064F90346002B01D00223D3E0FB6838
:101BE00093F83C30012B01D10223CCE0FB680122A9
:101BF00083F83C20FB681B681B6803F00103012B82
:101C000007D0FB681B681A68FB681B6842F001027A
:101C10001A60FB681B681A68FB681B6822F4006284
:101C20001A60FB68212283F83D20FB68102283F8AC
:101C30003E20FB6800221A64FB687A685A62FB68DF
:101C40003A895A85FB685B8D9AB2FB681A85FB68F6
:101C5000504ADA6279897B693A6AF86800F09CF840
:101C60000346002B01D001238DE000233B61FB687C
:101C70001B685B693B61FB681B689B693B613B6957
:101C800066E07A69396AF86800F022FA0346002BA8
:101C90000DD0FB681B6C042B07D1FB681B681A680E
:101CA000FB681B6842F400721A6001236BE0FB685A
:101CB0005B6A1A78FB681B681A61FB685B6A5A1CCE
:101CC000FB685A62FB685B8D9BB2013B9AB2FB6872
:101CD0005A85FB681B8D013B9AB2FB681A85FB682D
:101CE0001B685B6903F00403042B1BD1FB681B8D8D
:101CF000002B17D0FB685B6A1A78FB681B681A61B7
:101D0000FB685B6A5A1CFB685A62FB685B8D9BB27E
:101D1000013B9AB2FB685A85FB681B8D013B9AB266
:101D2000FB681A857A69396AF86800F019FA03467F
:101D3000002B0DD0FB681B6C042B07D1FB681B68C4
:101D40001A68FB681B6842F400721A6001231AE0EB
:101D5000FB681B8D002B94D1FB681B681A68FB681D
:101D60001B6842F400721A60FB68202283F83D2051
:101D7000FB68002283F83E20FB68002283F83C20A9
:101D8000002300E0022318461837BD4680BD00BF7F
:101D9000020010000000FFFF80B588B002AFF860BD
:101DA0007A603B600B467B81FB68DB6A7B617B6909
:101DB000082B06D07B69012B03D07B6913F5803F8C
:101DC00008D1FB681B681A68FB681B6842F48072C4
:101DD0001A600BE0FB681B6B122B07D1FB681B68BA
:101DE0001A68FB681B6842F480721A603B680093B3
:101DF0007B6800224FF00111F86800F04FF80346AD
:101E0000002B0DD0FB681B681B6803F48073B3F5CF
:101E1000807F03D1FB684FF400721A64032335E01E
:101E2000FB681B69B3F5804F08D17B89DBB21A468A
:101E3000FB681B6802F0FE021A611BE07B89DB1164
:101E4000DBB203F00603DBB263F00F03DAB2FB6828
:101E50001B681A613B687A680E49F86800F098F8C8
:101E60000346002B01D0012310E07B89DAB2FB6826
:101E70001B681A613B687A680749F86800F088F8BF
:101E80000346002B01D0012300E000231846183739
:101E9000BD4680BD080001000200010080B584B08D
:101EA00000AFF860B9603B601346FB7148E03B68E7
:101EB000B3F1FF3F44D0FFF793F90246BB69D31A51
:101EC0003A689A4202D33B68002B39D1BB681B0C9D
:101ED000DBB2012B0DD1FB681B685B69DA43BB6881
:101EE00013409BB2002B0CBF01230023DBB21A4628
:101EF0000CE0FB681B689B69DA43BB6813409BB22C
:101F0000002B0CBF01230023DBB21A46FB799A4257
:101F100016D1FB6800221A63FB68202283F83D205B
:101F2000FB68002283F83E20FB681B6C43F0200214
:101F3000FB681A64FB68002283F83C20012323E03D
:101F4000BB681B0CDBB2012B0DD1FB681B685B6906
:101F5000DA43BB6813409BB2002B0CBF0123002364
:101F6000DBB21A460CE0FB681B689B69DA43BB686E
:101F700013409BB2002B0CBF01230023DBB21A4697
:101F8000FB799A4293D0002318461037BD4680BD96
:101F900080B584B000AFF860B9607A603B6071E0F2
:101FA000FB681B685B6903F48063B3F5806F23D122
:101FB000FB681B681A68FB681B6842F400721A60B1
:101FC000FB681B686FF480625A61FB6800221A6329
:101FD000FB68202283F83D20FB68002283F83E2026
:101FE000FB681B6C43F00402FB681A64FB68002268
:101FF00083F83C20012367E07B68B3F1FF3F41D0C9
:10200000FFF7EEF802463B68D31A7A689A4202D389
:102010007B68002B36D1BB681B0CDBB2012B0CD1CB
:10202000FB681B685B69DA43BB6813409BB2002BFB
:1020300014BF01230023DBB20BE0FB681B689B6924
:10204000DA43BB6813409BB2002B14BF012300236B
:10205000DBB2002B16D0FB6800221A63FB6820223B
:1020600083F83D20FB68002283F83E20FB681B6C50
:1020700043F02002FB681A64FB68002283F83C20CE
:10208000012321E0BB681B0CDBB2012B0CD1FB68E8
:102090001B685B69DA43BB6813409BB2002B14BF1B
:1020A00001230023DBB20BE0FB681B689B69DA436A
:1020B000BB6813409BB2002B14BF01230023DBB28B
:1020C000002B7FF46DAF002318461037BD4680BD4E
:1020D00080B584B000AFF860B9607A6034E0F86829
:1020E00000F086F80346002B01D0012334E0BB68E2
:1020F000B3F1FF3F28D0FFF773F802467B68D31A8D
:10210000BA689A4202D3BB68002B1DD1FB681B68DA
:102110005B6903F08003802B16D0FB6800221A63F2
:10212000FB68202283F83D20FB68002283F83E20D4
:10213000FB681B6C43F02002FB681A64FB680022FA
:1021400083F83C20012307E0FB681B685B6903F010
:102150008003802BC3D1002318461037BD4680BDB5
:1021600080B584B000AFF860B9607A6034E0F86898
:1021700000F03EF80346002B01D0012334E0BB6899
:10218000B3F1FF3F28D0FFF72BF802467B68D31A44
:10219000BA689A4202D3BB68002B1DD1FB681B684A
:1021A0005B6903F00403042B16D0FB6800221A635A
:1021B000FB68202283F83D20FB68002283F83E2044
:1021C000FB681B6C43F02002FB681A64FB6800226A
:1021D00083F83C20012307E0FB681B685B6903F080
:1021E0000403042BC3D1002318461037BD4680BD1D
:1021F00080B483B000AF78607B681B685B6903F4D0
:102200008063B3F5806F1BD17B681B686FF48062BD
:102210005A617B6800221A637B68202283F83D2084
:102220007B68002283F83E207B681B6C43F004022D
:102230007B681A647B68002283F83C20012300E05D
:10224000002318460C37BD465DF8047B704780B408
:1022500083B000AF786039607B6893F83D30DBB2C3
:10226000202B29D17B68242283F83D207B681B68C2
:102270001A687B681B6822F001021A607B681B6881
:102280005A6A7B681B6822F010025A627B681B68DE
:10229000596A7B681B683A680A435A627B681B6804
:1022A0001A687B681B6842F001021A607B68202272
:1022B00083F83D20002300E0022318460C37BD467A
:1022C0005DF8047B704780B485B000AF78603960FA
:1022D0000023FB817B6893F83D30DBB2202B2AD1B1
:1022E0007B68242283F83D207B681B681A687B6822
:1022F0001B6822F001021A607B681B685B6AFB8125
:10230000FB8923F00F03FB813B689AB2FB891343DF
:10231000FB817B681B68FA895A627B681B681A68B4
:102320007B681B6842F001021A607B68202283F8F8
:102330003D20002300E0022318461437BD465DF817
:10234000047B704780B584B000AF786039607B68EB
:10235000002B01D10123CCE0684B1B6803F007037D
:102360003A689A420CD9654B3A68D2B21A70634BFC
:102370001B6803F007033A689A4201D00123B8E0D2
:102380007B681B6803F00203002B20D07B681B686E
:1023900003F00403002B05D0594B9B68584A43F4C3
:1023A000E05393607B681B6803F00803002B05D0A3
:1023B000534B9B68524A43F460439360504B9B6875
:1023C00023F0F0027B689B684D4913438B607B6868
:1023D0001B6803F00103002B44D07B685B68012B72
:1023E00007D1474B1B6803F40033002B19D101239D
:1023F0007FE07B685B68022B03D07B685B68032B04
:1024000007D13F4B1B6803F00073002B09D1012358
:102410006FE03B4B1B6803F00203002B01D101234B
:1024200067E0374B9B6823F003027B685B683449A5
:1024300013438B60FEF7D4FEF8600AE0FEF7D0FE8F
:102440000246FB68D31A41F28832934201D9032332
:102450004FE02B4B9B6803F00C027B685B689B0092
:102460009A42EBD1254B1B6803F007033A689A4266
:102470000CD2224B3A68D2B21A70204B1B6803F080
:1024800007033A689A4201D0012332E07B681B6857
:1024900003F00403002B08D0194B9B6823F4E0528F
:1024A0007B68DB68164913438B607B681B6803F00D
:1024B0000803002B09D0124B9B6823F460427B6811
:1024C0001B69DB000E4913438B6000F021F80246C4
:1024D0000B4B9B681B0903F00F030A49CB5C22FAE4
:1024E00003F3094A1360094B1B681846FEF734FED4
:1024F000002318461037BD4680BD00BF003C024097
:1025000000380240A04500082000002024000020E0
:102510002DE9B04F94B000AF00237B640023FB642F
:1025200000233B640023BB64794B9B6803F00C03DE
:10253000082B0DD0082B00F2E180002B02D0042BD9
:1025400003D0DBE0734BBB64DBE0734BBB64D8E0D0
:102550006F4B5B6803F03F037B646D4B5B6803F478
:102560008003002B63D06A4B5B689B090022BB632E
:10257000FA63BB6BC3F308033B6300237B63D7E9B8
:102580000C4522462B464FF000004FF00001590148
:1025900041EAD261500102460B462146511A396187
:1025A000294663EB01037B614FF000024FF000030B
:1025B000D7E904AB59468B01514643EA9163514632
:1025C0008A015146B2EB0108594663EB01094FF00D
:1025D00000024FF000034FEAC90343EA58734FEA81
:1025E000C80290469946234618EB0303BB602B466E
:1025F00049EB0303FB604FF000024FF00003D7E903
:10260000024529464B02214643EAD15321464A025C
:10261000104619467B6C0022BB62FA62D7E90A2396
:10262000FDF756FE02460B461346FB6458E0384B56
:102630005B689B09002218461146C0F308033B6201
:1026400000237B62D7E9088942464B464FF00000E1
:102650004FF00001590141EAD261500102460B4698
:102660004146B2EB010A494663EB010B4FF0000211
:102670004FF000034FEA8B1343EA9A634FEA8A1242
:10268000B2EB0A0463EB0B054FF000024FF00003BE
:10269000EB0043EA5473E20014461D464346E31838
:1026A0003B604B4645EB03037B604FF000024FF06D
:1026B0000003D7E9004529468B02214643EA91539E
:1026C00021468A02104619467B6C0022BB61FA61E2
:1026D000D7E90623FDF7FCFD02460B461346FB64D3
:1026E0000B4B5B681B0C03F0030301335B003B6483
:1026F000FA6C3B6CB2FBF3F3BB6402E0054BBB64CA
:1027000000BFBB6C18465037BD46BDE8B08F00BF58
:10271000003802400024F40000127A0080B400AFB8
:10272000034B1B681846BD465DF8047B704700BF2D
:102730002000002080B500AFFFF7F0FF0246054BF8
:102740009B689B0A03F007030349CB5C22FA03F35F
:10275000184680BD00380240B045000880B500AF83
:10276000FFF7DCFF0246054B9B685B0B03F007039A
:102770000349CB5C22FA03F3184680BD00380240BF
:10278000B045000880B586B000AF78607B68002B4C
:1027900001D1012373E27B681B6803F00103002B66
:1027A00075D0884B9B6803F00C03042B0CD0854B31
:1027B0009B6803F00C03082B12D1824B5B6803F477
:1027C0008003B3F5800F0BD17E4B1B6803F40033FD
:1027D000002B5BD07B685B68002B57D101234EE256
:1027E0007B685B68B3F5803F06D1764B1B68754A02
:1027F00043F4803313601DE07B685B68B3F5A02F62
:102800000CD1704B1B686F4A43F4802313606D4BEF
:102810001B686C4A43F4803313600BE0694B1B6800
:10282000684A23F480331360664B1B68654A23F4BF
:10283000802313607B685B68002B13D0FEF7D0FC0D
:10284000386108E0FEF7CCFC02463B69D31A642BE2
:1028500001D9032313E25B4B1B6803F40033002B05
:10286000F0D014E0FEF7BCFC386108E0FEF7B8FCDD
:1028700002463B69D31A642B01D90323FFE1514B74
:102880001B6803F40033002BF0D100E000BF7B682D
:102890001B6803F00203002B63D04A4B9B6803F0D4
:1028A0000C03002B0BD0474B9B6803F00C03082B49
:1028B0001CD1444B5B6803F48003002B16D1414BC1
:1028C0001B6803F00203002B05D07B68DB68012B3B
:1028D00001D00123D3E13B4B1B6823F0F8027B6856
:1028E0001B69DB00374913430B603AE07B68DB6808
:1028F000002B20D0344B01221A60FEF771FC3861A6
:1029000008E0FEF76DFC02463B69D31A022B01D9A1
:102910000323B4E12B4B1B6803F00203002BF0D020
:10292000284B1B6823F0F8027B681B69DB002549F4
:1029300013430B6015E0244B00221A60FEF750FC95
:10294000386108E0FEF74CFC02463B69D31A022BC3
:1029500001D9032393E11B4B1B6803F00203002BF7
:10296000F0D17B681B6803F00803002B36D07B682E
:102970005B69002B16D0154B01221A60FEF730FC64
:10298000386108E0FEF72CFC02463B69D31A022BA3
:1029900001D9032373E10B4B5B6F03F00203002BA0
:1029A000F0D01BE0094B00221A60FEF719FC3861D9
:1029B0000EE0FEF715FC02463B69D31A022B07D93D
:1029C00003235CE10038024000004742800E47428A
:1029D0008A4B5B6F03F00203002BEAD17B681B6814
:1029E00003F00403002B00F097800023FB75834B5A
:1029F0001B6C03F08053002B0FD10023BB607F4B77
:102A00001B6C7E4A43F0805313647C4B1B6C03F0B9
:102A10008053BB60BB680123FB75794B1B6803F4D3
:102A20008073002B18D1764B1B68754A43F4807372
:102A30001360FEF7D5FB386108E0FEF7D1FB0246D4
:102A40003B69D31A022B01D9032318E16C4B1B6895
:102A500003F48073002BF0D07B689B68012B06D1B8
:102A6000664B1B6F654A43F0010313671CE07B68EC
:102A70009B68052B0CD1614B1B6F604A43F004032C
:102A800013675E4B1B6F5D4A43F0010313670BE056
:102A90005A4B1B6F594A23F001031367574B1B6FA7
:102AA000564A23F0040313677B689B68002B15D0FC
:102AB000FEF796FB38610AE0FEF792FB02463B699F
:102AC000D31A41F28832934201D90323D7E04B4B0A
:102AD0001B6F03F00203002BEED014E0FEF780FB27
:102AE00038610AE0FEF77CFB02463B69D31A41F2EB
:102AF0008832934201D90323C1E0404B1B6F03F09E
:102B00000203002BEED1FB7D012B05D13B4B1B6C4F
:102B10003A4A23F0805313647B689B69002B00F0D2
:102B2000AD80364B9B6803F00C03082B60D07B68AC
:102B30009B69022B45D1334B00221A60FEF750FBF4
:102B4000386108E0FEF74CFB02463B69D31A022BC2
:102B500001D9032393E0294B1B6803F00073002B7A
:102B6000F0D17B68DA697B681B6A1A437B685B6A11
:102B70009B011A437B689B6A5B08013B1B041A4359
:102B80007B68DB6A1B061A437B681B6B1B071B49B0
:102B900013434B601B4B01221A60FEF721FB386187
:102BA00008E0FEF71DFB02463B69D31A022B01D950
:102BB000032364E0114B1B6803F00073002BF0D07B
:102BC0005CE0104B00221A60FEF70AFB386108E057
:102BD000FEF706FB02463B69D31A022B01D90323F9
:102BE0004DE0064B1B6803F00073002BF0D145E06D
:102BF0007B689B69012B07D1012340E0003802402C
:102C000000700040600047421F4B5B68FB607B68C0
:102C10009B69012B30D0FB6803F480027B68DB6981
:102C20009A4229D1FB6803F03F027B681B6A9A42F3
:102C300022D1FA6847F6C07313407A68526A92014B
:102C4000934219D1FB6803F440327B689B6A5B08AE
:102C5000013B1B049A420FD1FB6803F070627B6852
:102C6000DB6A1B069A4207D1FB6803F0E0427B68EF
:102C70001B6B1B079A4201D0012300E0002318467A
:102C80001837BD4680BD00BF0038024080B582B015
:102C900000AF78607B68002B01D1012342E07B68A4
:102CA00093F84130DBB2002B06D17B68002283F819
:102CB00040207868FEF732F97B68242283F84120AF
:102CC0007B681B68DA687B681B6822F40052DA6054
:102CD000786800F0BBFC7B681B681A697B681B681E
:102CE00022F490421A617B681B685A697B681B68F2
:102CF00022F02A025A617B681B68DA687B681B68CD
:102D000042F40052DA607B6800225A647B68202219
:102D100083F841207B68202283F842207B680022D0
:102D20005A63002318460837BD4680BD80B485B07D
:102D300000AFF860B9601346FB80FB6893F8413040
:102D4000DBB2202B21D1BB68002B02D0FB88002BEB
:102D500001D101231AE0FB68BA681A62FB68FA889D
:102D60009A84FB68FA88DA84FB6800225A64FB685C
:102D7000212283F84120FB681B68DA68FB681B6826
:102D800042F08002DA60002300E002231846143784
:102D9000BD465DF8047B704780B5BAB000AF78607F
:102DA0007B681B681B68C7F8E4307B681B68DB68BE
:102DB000C7F8E0307B681B685B69C7F8DC3000232C
:102DC000C7F8D8300023C7F8D430D7F8E43003F080
:102DD0000F03C7F8D830D7F8D830002B0FD1D7F869
:102DE000E43003F02003002B09D0D7F8E03003F0E3
:102DF0002003002B03D0786800F069FB5BE2D7F872
:102E0000D830002B00F0DE80D7F8DC3003F001036F
:102E1000002B06D1D7F8E03003F49073002B00F0BC
:102E2000D180D7F8E43003F00103002B0BD0D7F8A2
:102E3000E03003F48073002B05D07B685B6C43F0BB
:102E400001027B685A64D7F8E43003F00403002BD6
:102E50000BD0D7F8DC3003F00103002B05D07B68E2
:102E60005B6C43F002027B685A64D7F8E43003F0ED
:102E70000203002B0BD0D7F8DC3003F00103002B4A
:102E800005D07B685B6C43F004027B685A64D7F81A
:102E9000E43003F00803002B11D0D7F8E03003F042
:102EA0002003002B05D1D7F8DC3003F00103002B01
:102EB00005D07B685B6C43F008027B685A647B68D2
:102EC0005B6C002B00F0F281D7F8E43003F02003B4
:102ED000002B08D0D7F8E03003F02003002B02D0FD
:102EE000786800F0F4FA7B681B685B6903F04003C4
:102EF000402B0CBF01230023DBB2C7F8D4307B6822
:102F00005B6C03F00803002B03D1D7F8D430002BFF
:102F10004FD0786800F0FCF97B681B685B6903F0B0
:102F20004003402B41D17B681B681433C7F89C30A9
:102F3000D7F89C3053E8003FC7F89830D7F898305E
:102F400023F04003C7F8D0307B681B681433D7F8F0
:102F5000D020C7F8A820C7F8A430D7F8A410D7F815
:102F6000A82041E80023C7F8A030D7F8A030002BF4
:102F7000D9D17B68DB6B002B13D07B68DB6B7E4A7F
:102F80001A657B68DB6B1846FEF7DBFA0346002BFD
:102F900016D07B68DB6B1B6D7A68D26B1046984746
:102FA0000EE0786800F09EF90AE0786800F09AF97F
:102FB00006E0786800F096F97B6800225A6475E1B3
:102FC00000BF73E17B681B6B012B40F04F81D7F88A
:102FD000E43003F01003002B00F04881D7F8E03014
:102FE00003F01003002B00F041810023BB607B68DD
:102FF0001B681B68BB607B681B685B68BB60BB6849
:103000007B681B685B6903F04003402B40F0B6808F
:103010007B68DB6B1B685B68A7F8BE30B7F8BE3017
:10302000002B00F045817B689B8DB7F8BE209A424B
:1030300080F03E817B68B7F8BE20DA857B68DB6B69
:10304000DB69B3F5807F00F088807B681B680C33F8
:10305000C7F88830D7F8883053E8003FC7F8843085
:10306000D7F8843023F48073C7F8B8307B681B68C6
:103070000C33D7F8B820C7F89420C7F89030D7F8A9
:103080009010D7F8942041E80023C7F88C30D7F887
:103090008C30002BD9D17B681B6814337B677B6F26
:1030A00053E8003F3B673B6F23F00103C7F8B430A0
:1030B0007B681B681433D7F8B420C7F88020FB67FF
:1030C000F96FD7F8802041E80023BB67BB6F002B66
:1030D000E1D17B681B6814333B663B6E53E8003FCD
:1030E000FB65FB6D23F04003C7F8B0307B681B68BD
:1030F0001433D7F8B020FA66BB66B96EFA6E41E8B1
:1031000000237B667B6E002BE3D17B68202283F853
:1031100042207B6800221A637B681B680C33FB64C7
:10312000FB6C53E8003FBB64BB6C23F01003C7F893
:10313000AC307B681B680C33D7F8AC20BA657B6574
:10314000796DBA6D41E800233B653B6D002BE3D1FF
:103150007B68DB6B1846FEF784F97B6802225A63B2
:103160007B689A8D7B68DB8D9BB2D31A9BB2194624
:10317000786800F0C1F89BE0D73300087B689A8D2F
:103180007B68DB8D9BB2D31AA7F8CE307B68DB8DD2
:103190009BB2002B00F08E80B7F8CE30002B00F0F1
:1031A00089807B681B680C33BB63BB6B53E8003FB3
:1031B0007B637B6B23F49073C7F8C8307B681B6814
:1031C0000C33D7F8C8207A643B64396C7A6C41E8D8
:1031D0000023FB63FB6B002BE3D17B681B6814337C
:1031E0007B627B6A53E8003F3B623B6A23F001034A
:1031F000C7F8C4307B681B681433D7F8C4203A631F
:10320000FB62F96A3A6B41E80023BB62BB6A002BA0
:10321000E3D17B68202283F842207B6800221A6376
:103220007B681B680C333B613B6953E8003FFB60E4
:10323000FB6823F01003C7F8C0307B681B680C33B1
:10324000D7F8C020FA61BB61B969FA6941E8002387
:103250007B617B69002BE3D17B6802225A63B7F85C
:10326000CE301946786800F047F823E0D7F8E4300C
:1032700003F08003002B09D0D7F8E03003F080037F
:10328000002B03D0786800F0BAF814E0D7F8E430E7
:1032900003F04003002B0ED0D7F8E03003F04003DA
:1032A000002B08D0786800F0FAF804E000BF02E0D4
:1032B00000BF00E000BFE837BD4680BD80B483B0EA
:1032C00000AF786000BF0C37BD465DF8047B7047E7
:1032D00080B483B000AF786000BF0C37BD465DF8A6
:1032E000047B704780B483B000AF786000BF0C37B8
:1032F000BD465DF8047B704780B483B000AF786052
:103300000B467B8000BF0C37BD465DF8047B7047E1
:1033100080B495B000AF78607B681B680C337B632A
:103320007B6B53E8003F3B633B6B23F49073FB6480
:103330007B681B680C33FA6C3A64FB63F96B3A6C7C
:1033400041E80023BB63BB6B002BE5D17B681B68A6
:1033500014333B623B6A53E8003FFB61FB6923F097
:103360000103BB647B681B681433BA6CFA62BB62EE
:10337000B96AFA6A41E800237B627B6A002BE5D1D7
:103380007B681B6B012B19D17B681B680C33FB60BE
:10339000FB6853E8003FBB60BB6823F010037B640D
:1033A0007B681B680C337A6CBA617B617969BA6996
:1033B00041E800233B613B69002BE5D17B6820227B
:1033C00083F842207B6800221A6300BF5437BD4651
:1033D0005DF8047B704780B584B000AF78607B688F
:1033E0009B6BFB60FB680022DA85FB680022DA84B5
:1033F000F868FFF777FF00BF1037BD4680BD80B487
:1034000085B000AF78607B6893F84130DBB2212B48
:103410003ED17B689B68B3F5805F14D17B681B69E4
:10342000002B10D17B681B6AFB60FB681B881A4667
:103430007B681B68C2F308025A607B681B6A9A1C8F
:103440007B681A6208E07B681B6A591C7A68116203
:103450001A787B681B685A607B68DB8C9BB2013BE7
:103460009BB27A681946D184002B0FD17B681B6808
:10347000DA687B681B6822F08002DA607B681B6870
:10348000DA687B681B6842F04002DA60002300E0E3
:10349000022318461437BD465DF8047B704780B59B
:1034A00082B000AF78607B681B68DA687B681B6855
:1034B00022F04002DA607B68202283F8412078689D
:1034C000FFF7FCFE002318460837BD4680BD80B5D7
:1034D0008CB000AF78607B6893F84230DBB2222B6F
:1034E00040F0AE807B689B68B3F5805F17D17B6846
:1034F0001B69002B13D10023FB627B689B6ABB62B4
:103500007B681B685B689BB2C3F308039AB2BB6A13
:103510001A807B689B6A9A1C7B689A6226E07B68AB
:103520009B6AFB620023BB627B689B68B3F5805F8C
:1035300007D07B689B68002B0AD17B681B69002B36
:1035400006D17B681B685B68DAB2FB6A1A7008E018
:103550007B681B685B68DBB203F07F03DAB2FB6A4F
:103560001A707B689B6A5A1C7B689A627B68DB8D49
:103570009BB2013B9BB27A681946D185002B5DD185
:103580007B681B68DA687B681B6822F02002DA60BF
:103590007B681B68DA687B681B6822F48072DA60DB
:1035A0007B681B685A697B681B6822F001025A61BC
:1035B0007B68202283F842207B6800225A637B6864
:1035C0001B6B012B35D17B6800221A637B681B685B
:1035D0000C337B617B6953E8003F3B613B6923F01F
:1035E00010037B627B681B680C337A6A3A62FB616A
:1035F000F9693A6A41E80023BB61BB69002BE5D158
:103600007B681B681B6803F01003102B0AD1002392
:10361000FB607B681B681B68FB607B681B685B68E2
:10362000FB60FB687B689B8D19467868FFF764FE3A
:1036300002E07868FFF74CFE002302E0002300E080
:10364000022318463037BD4680BD00002DE9B04F3B
:10365000C0B000AFC7F8F400D7F8F4301B681B699E
:1036600023F44050D7F8F430D968D7F8F4301A680A
:1036700040EA01031361D7F8F4309A68D7F8F430C0
:103680001B691A43D7F8F4305B691A43D7F8F43052
:10369000DB691343C7F8F830D7F8F4301B68DB68F0
:1036A00023F4164121F00C01D7F8F4301A68D7F84A
:1036B000F8300B43D360D7F8F4301B685B6923F410
:1036C0004070D7F8F4309969D7F8F4301A6840EAB6
:1036D00001035361D7F8F4301A68954B9A4211D020
:1036E000D7F8F4301A68934B9A420BD0D7F8F430DD
:1036F0001A68914B9A4205D0D7F8F4301A688F4B6C
:103700009A4204D1FFF72AF8C7F8FC0003E0FFF75C
:1037100011F8C7F8FC00D7F8F430DB69B3F5004FB7
:1037200040F01081D7F8FC300022C7F8E830C7F825
:10373000EC20D7E93A4522462B469118B9655B4102
:10374000FB65D7E91623214612EB0108294643EB16
:1037500001094FF000024FF000034FEAC90343EAAA
:1037600058734FEAC80290469946234618EB030364
:10377000C7F8E0302B4649EB0303C7F8E430D7F82D
:10378000F4305B680022C7F8D830C7F8DC20D7E9EE
:1037900036120B46DB183B65134642EB03037B6591
:1037A000D7E91423D7E93801FCF792FD02460B460E
:1037B000634BA3FB02235B091C01D7F8FC300022FA
:1037C000C7F8D030C7F8D420D7E9348942464B46F1
:1037D0009118B9645B41FB64D7E91223414612EBAF
:1037E000010A494643EB010B4FF000024FF0000382
:1037F0004FEACB0343EA5A734FEACA0292469B460A
:1038000043461AEB0303C7F8C8304B464BEB0303A0
:10381000C7F8CC30D7F8F4305B680022C7F8C03066
:10382000C7F8C420D7E930120B46DB183B641346B7
:1038300042EB03037B64D7E91023D7E93201FCF79D
:1038400047FD02460B4611463D4BA3FB01235B0996
:10385000642202FB03F3CB1ADB0003F13202384B84
:10386000A3FB02235B095B0003F4F8731C44D7F845
:10387000FC300022C7F8B830C7F8BC20D7E92E8941
:1038800042464B469118B9635B41FB63D7E90E236F
:1038900041465118396349464B417B634FF0000262
:1038A0004FF00003D7E90CAB5946CB00514643EA31
:1038B00051735146CA0010461946034642469B18AA
:1038C000C7F8B0304B460A4642EB0303C7F8B430A2
:1038D000D7F8F4305B680022C7F8A830C7F8AC20EE
:1038E000D7E92A120B46DB18BB62134642EB0303EF
:1038F000FB62D7E90A23D7E92C01FCF7E9FC024671
:103900000B460F4BA3FB02135B09642101FB03F37E
:10391000D31ADB0032330A4AA2FB03235B0903F00C
:103920000702D7F8F4301B6822449A600AE100BF0E
:10393000001001400014014000180140001C01402B
:103940001F85EB51D7F8FC300022C7F8A030C7F82C
:10395000A420D7E9288942464B46911839625B4139
:103960007B62D7E9082341465418494643EB0105D9
:103970004FF000024FF00003EB0043EA5473E20003
:1039800014461D464346E318C7F898304B4645EBAE
:103990000303C7F89C30D7F8F4305B680022C7F8FF
:1039A0009030C7F894204FF000024FF00003D7E9A1
:1039B000244529468B00214643EA917321468A001B
:1039C000D7E92601FCF784FC02460B46604BA3FBBB
:1039D00002235B091C01D7F8FC300022C7F88830AD
:1039E000C7F88C20D7E9228942464B469118B96125
:1039F0005B41FB61D7E906234146511839614946CD
:103A00004B417B614FF000024FF00003D7E904AB5C
:103A10005946CB00514643EA51735146CA001046FD
:103A20001946034642469B18C7F880304B460A4663
:103A300042EB0303C7F88430D7F8F4305B68002208
:103A4000BB67FA674FF000024FF00003D7E91E8909
:103A500049468B00414643EA917341468A00D7E9C3
:103A60002001FCF735FC02460B461146384BA3FB00
:103A700001235B09642202FB03F3CB1A1B013233DF
:103A8000334AA2FB03235B0903F0F0031C44D7F87D
:103A9000FC3000223B677A67D7E91C8942464B46D7
:103AA0009118B9605B41FB60D7E902234146511888
:103AB000396049464B417B604FF000024FF00003F4
:103AC000D7E900AB5946CB00514643EA5173514602
:103AD000CA0010461946034642469B18BB664B4631
:103AE0000A4642EB0303FB66D7F8F4305B6800221A
:103AF0003B667A664FF000024FF00003D7E9188961
:103B000049468B00414643EA917341468A00D7E912
:103B10001A01FCF7DDFB02460B460D4BA3FB02131B
:103B20005B09642101FB03F3D31A1B013233084AFA
:103B3000A2FB03235B0903F00F02D7F8F4301B68E4
:103B400022449A6000BF07F58077BD46BDE8B08F7C
:103B50001F85EB510CB430B5174B0C1E1D689DB082
:103B600008DA8B232B604FF0FF301DB0BDE83040EA
:103B700002B070474FF40273ADF8143014BF04F173
:103B8000FF332346049307934FF6FF73029006908A
:103B9000ADF81630209A21AB02A92846019300F017
:103BA000CFF9431CBCBF8B232B60002CDDD0029BC4
:103BB00000221A70D9E700BF2C00002030B514464F
:103BC000002C9BB005461A4605DA8B2303604FF0A4
:103BD000FF301BB030BD4FF40273ADF80C3014BF92
:103BE00004F1FF332346029305934FF6FF730091D0
:103BF0000491ADF80E3069461E9B00F0A1F9431CFC
:103C0000BCBF8B232B60002CE3D0009B00221A70DA
:103C1000DFE7000007B5009313460A460146034854
:103C20000068FFF7CBFF03B05DF804FB2C00002019
:103C300002440346934200D1704703F8011BF9E7A1
:103C4000014B1868704700BF2C00002070B50D4D67
:103C50000D4C641BA4100026A64209D10B4D0C4C40
:103C600000F066FC641BA4100026A64205D170BDBE
:103C700055F8043B98470136EEE755F8043B984762
:103C80000136F2E7F4450008F4450008F445000861
:103C9000F84500087047704738B50546002941D0FF
:103CA00051F8043C0C1F002BB8BFE41800F0E0F8FA
:103CB0001D4A136833B9636014602846BDE8384074
:103CC00000F0DCB8A34208D9206821188B4201BF5C
:103CD00019685B6809182160EDE71A465B680BB14B
:103CE000A342FAD911685018A0420BD120680144B0
:103CF000501883421160E0D118685B685360084433
:103D00001060DAE702D90C232B60D6E7206821186F
:103D10008B4204BF19685B68636004BF09182160A7
:103D20005460CAE738BD00BF980E002070B50F4E32
:103D30000C463168054611B900F0A6FB30602146FB
:103D4000284600F0A1FB431C03D14FF0FF3420466E
:103D500070BDC41C24F00304A042F8D0211A2846E8
:103D600000F092FB0130F2D1EFE700BF940E00208B
:103D70002DE9F843CD1C25F0030508350C2D38BF7F
:103D80000C25002D064601DBA94204D90C23336023
:103D90000020BDE8F883DFF8D48000F069F8D8F897
:103DA00000301C4644BB29463046FFF7BFFF431C8A
:103DB000044658D1D8F800402746002F43D1002CA4
:103DC0004BD023683946304604EB030900F05CFB16
:103DD000814542D121686D1A29463046FFF7A6FF7A
:103DE00001303AD023682B442360D8F800305A6859
:103DF00062BBC8F800700FE02268521B20D40B2A67
:103E000017D96119A342256018BF5960636808BFBC
:103E1000C8F8001062514B60304600F02FF804F1F2
:103E20000B00231D20F00700C21A1CBF1B1AA35051
:103E3000AFE76268A3420CBFC8F800205A60EBE706
:103E400023466468AEE73C467F68B6E71A465B687F
:103E5000A342FBD100235360DEE70C2333603046DE
:103E600000F00CF894E70560D6E700BF980E00203C
:103E70000148FFF70FBF00BF900E00200148FFF779
:103E80000ABF00BF900E00202DE9F0478E681F4644
:103E9000BE420B6882460C4690462DD8B1F90C20E4
:103EA00012F4906F26D06569096905EB4505A3EB0F
:103EB000010905EBD5757B1C4B446D109D4238BF45
:103EC0001D46530527D52946FFF752FF064660B326
:103ED00021694A4600F0E8FAA38923F4906343F08D
:103EE0008003A381266165614E44A5EB0905266028
:103EF000A5603E46BE4200D93E4620683246414655
:103F000000F0A8FAA3689B1BA360236833442360D6
:103F10000020BDE8F0872A4600F0D4FA06460028C3
:103F2000E0D121695046FFF7B7FE0C23CAF80030F4
:103F3000A38943F04003A3814FF0FF30E9E700007D
:103F40002DE9F04F98468B891B069DB007460D461C
:103F5000144610D50B6973B94021FFF709FF28609B
:103F6000286130B90C233B604FF0FF301DB0BDE835
:103F7000F08F40236B610023099320238DF82930B3
:103F8000CDF80C803023DFF89C818DF82A304FF07B
:103F9000010923469A4613F8012B0AB1252AF9D1C3
:103FA000BAEB040B0BD05B46224629463846FFF796
:103FB0006BFF013000F0A780099A5A4409929AF8E1
:103FC0000030002B00F09F8000234FF0FF32CDE93E
:103FD00005230AF1010A049307938DF853301A93CD
:103FE0005446052214F8011B4E48FCF721F9049AA7
:103FF000D8B9D00644BF20238DF85330110744BFF1
:104000002B238DF853309AF800302A2B15D0079ABD
:10401000544600204FF00A0C214611F8013B303B7A
:10402000092B4BD9B0B1079214E0A0EB080309FAB1
:1040300003F313430493A246D2E7039B191D1B68A5
:104040000391002BBBBF5B4242F002020793079330
:10405000B8BF049223782E2B0AD163782A2B32D151
:10406000039B1A1D1B68039243EAE3730234059312
:10407000DFF8C0A0217803225046FCF7D9F838B108
:10408000049BA0EB0A0040228240134301340493B6
:1040900014F8011B24488DF828100622FCF7C8F8F4
:1040A000002836D0214B1BBB039B073323F00703AB
:1040B00008330393099B334409936AE70CFB0232EC
:1040C0000C460120A8E700230134059319464FF060
:1040D0000A0C204610F8012B303A092A03D9002B8C
:1040E000C6D00591C4E70CFB012104460123F0E78B
:1040F00003AB00932A460E4B04A93846AFF3008069
:10410000421C0646D6D1AB895B063FF52DAF099818
:104110002CE703AB00932A46054B04A9384600F070
:1041200079F8EDE7B8450008C24500080000000036
:10413000893E0008BE4500082DE9F047164698461E
:104140008A680B69DDF820909342B8BF134633604C
:1041500091F8432007460C460AB1013333602368C7
:10416000990642BF336802333360256815F00605AF
:1041700006D104F1190AE36832689B1AAB4226DCC7
:1041800094F843302268003B18BF012392062BD4D9
:1041900004F1430241463846C84701301ED0236827
:1041A000226903F00603042B02BFE5683368ED1AA9
:1041B000A3680CBF25EAE57500259342C4BF9B1A8E
:1041C000ED1800261A34B5421AD1002008E0012368
:1041D000524641463846C847013003D14FF0FF30C0
:1041E000BDE8F0870135C6E7E1185A1C302081F898
:1041F0004300224494F8451082F843100233C7E785
:104200000123224641463846C8470130E6D00136F0
:10421000D9E700002DE9FF470F7E0C9E782F9146CD
:1042200080460C469A4601F1430207D8622F0AD80D
:10423000002F00F0D280582F00F0B98004F1420620
:1042400084F842703AE0A7F16303152BF6D801A178
:1042500051F823F0AD420008C14200083D42000879
:104260003D4200083D4200083D420008C1420008AE
:104270003D4200083D4200083D4200083D42000822
:10428000C1430008EB4200087B4300083D420008A0
:104290003D420008E34300083D420008EB420008AD
:1042A0003D4200083D4200088343000833681A1D60
:1042B0001B68326004F1420684F8423001239DE01D
:1042C00033682068191D3160060601D51D6803E0BA
:1042D0004506FBD5B3F90050002D03DA2D236D42BE
:1042E00084F8433059480A2311E0216833680806EE
:1042F00053F8045B02D4490648BFADB26F2F534850
:10430000336014BF0A230823002184F84310666831
:10431000A660002EA2BF216821F0040121600DB922
:10432000002E4BD01646B5FBF3F103FB1157C75DCA
:1043300006F8017D2F46BB420D46F4D9082B0BD160
:104340002368DF0708D5236961689942DEBF3023FF
:1043500006F8013C06F1FF36921B2261CDF800A061
:104360004B4603AA21464046FFF7E6FE01304AD1FC
:104370004FF0FF3004B0BDE8F087236843F020031E
:1043800023603348782784F84570236831681F0616
:1043900051F8045B02D45F0648BFADB23160D90763
:1043A00044BF43F0200323601DB11023ACE727482E
:1043B000E9E7236823F020032360F6E71646BDE70C
:1043C000336825686169181D30602E061B6801D5A9
:1043D000196002E06806FBD51980002323611646A8
:1043E000BCE733681A1D32601E68626800213046DF
:1043F000FBF71EFF08B1801B606063682361002328
:1044000084F84330AAE72369324649464046D047FC
:104410000130ADD023689B0713D4E068039B98421A
:10442000B8BF1846A6E70123324649464046D04762
:1044300001309DD00135E36803995B1AAB42F2DC91
:10444000EBE7002504F11906F5E700BFC9450008B0
:10445000DA450008884210B501EB020402D9844213
:10446000234607D8431EA14208D011F8012B03F8B8
:10447000012FF8E7024401468A4200D110BD13F82B
:10448000014D02F8014DF7E738B5064D002304460B
:1044900008462B60FCF7CCFD431C02D12B6803B10E
:1044A000236038BD8C0E00200A44914200F1FF3396
:1044B00000D1704710B511F8014B03F8014F91423C
:1044C000F9D110BD2DE9F041804615460C4621B9C1
:1044D000BDE8F0411146FFF74BBC2AB9FFF7DCFB02
:1044E00000242046BDE8F08100F01AF88542064617
:1044F00002D8B5EB500FF4D829464046FFF738FCF8
:1045000007460028ECD0B5422A46214628BF32464D
:10451000FFF7CAFF21464046FFF7BEFB3C46E0E7F7
:1045200051F8043C181F002BBCBF0B58C018704733
:10453000F8B500BFF8BC08BC9E467047F8B500BF90
:08454000F8BC08BC9E46704760
:104548005B44454255475D005B494E464F5D000060
:104558005B5741524E5D00005B4552524F525D0021
:104568005B464154414C5D005B414C4C5D00000092
:104578002573093A200000000D0A0000686969697E
:1045880020686565656C6C6C6F6F6F6F6F6F6F2EF1
:104598002E2E2E2E0000000000000000000000005B
:1045A80001020304060708090000000001020304D1
:1045B800232D302B2000686C4C0065666745464704
:1045C8000030313233343536373839414243444587
:1045D80046003031323334353637383961626364F6
:0445E8006566000004
:0845EC0034BCFF7F0100000058
:0445F40005020008B4
:0445F800E1010008D5
:1045FC0001000000484500085045000858450008D7
:10460C00604500086845000870450008010100007D
:10461C000024F40010000000010000003000002015
:10462C0000000000540D0020BC0D0020240E0020C2
:10463C00000000000000000000000000000000006E
:10464C00000000000000000000000000000000005E
:10465C00000000000000000000000000000000004E
:0C466C0000000000000000000000000042
:04000005080010C11E
:00000001FF
